:10000000830101308A004A29F20003088301C800F5
:100010000408C9007008CB007108CA0083120313DA
:100020000C1C202883160C1C1F2883120C1083160E
:100030000C108312A801A901A601043097008312B5
:100040000C1DC5280C11BE281608AB001508AA0007
:10005000B9281608F100F0011508F0042A0870020A
:10006000AA002B08031C2B0A7102AB0001302B02E3
:10007000B13003192A020318442800302B02AC3097
:1000800003192A0203184B28A801A901A60104306C
:1000900097000C11C5280A3097001608AD00150806
:1000A000AC002B08F1002A08F0000310F10CF00C52
:1000B0007008AC070318AD0A7108AD072B08F100F2
:1000C0002A08F0000310F10CF00C7008AA070318BE
:1000D000AB0A7108AB072D0896002C089500BB28C9
:1000E000261C9E2826081B3A031D8928A91D7D2849
:1000F00020188128201520148128201C81282015F3
:1001000020102808A700A801A901A6010430970023
:100110009B28A60A1608AD001508AC002A08AC07F3
:100120000318AD0A2B08AD070A3097002D0896007A
:100130002C0895000C1183160C10C52810108F0187
:100140008E0183160C1483120C101014861DB62811
:100150002908F1002808F0000310F00DF10D01301E
:100160007004A8007108A9000430BA280310A80D73
:10017000A90D053097000C11A60AC52826080319F9
:100180002428013A0319292870280B1D00290B1176
:100190008312A40A24080A3A031DDE281F308500B2
:1001A0000F308500F0308600A401A10A2108220644
:1001B000031DE628A1010230A006E6280F308500C5
:1001C000F130860000000000F0308600A01CEF280F
:1001D00024082E3E840083130008C700F028C701BE
:1001E0002408383E84008313000847040F39850033
:1001F0002408383E8400831300084704F039860041
:1002000083128C1E2529981C0A298316A014831298
:1002100018121816181D0F298316201483121A0895
:10022000C6008316220A03398312C7008316A20070
:1002300083124708831623060319A0148312470864
:10024000A63E84008313460880000C1E3D298316B9
:100250000C1E3D292408250603193C29250A0339CB
:100260008312C7008316A50083124708AA3E8400A4
:100270008313000899003D290C12031383124B08C5
:10028000F0004A08F1004908840048088300F20E93
:10029000720E09002030840021305F21213084005B
:1002A00048305F21A0308400A1305F21A13084005C
:1002B000B6305F218301102B04068001840A0406F6
:1002C000031D5C29003482073F3406347A346E34CF
:1002D00047346D347D3426347F346F3477345D3465
:0802E00039345E3479347134C5
:1005660083160313A10183120800831603132208BE
:1005760023060030031D0130831208008312031383
:10058600420883169B001C141A088312080083165F
:100596000313220823060319CC2A230A03398312DC
:1005A600C4008316A30083124408A63E8400831366
:1005B6000008080083120313420883169B00831267
:1005C600440883169A001C158B1355309D00AA30DB
:1005D6009D009C148B1783128C1FEF2A83161C1107
:1005E60083128C13080083120313C4008316240A93
:1005F60003398312C500450883162506831203199D
:10060600FE2A4508AA3E8400831344088000450854
:100616008316A4000C1683120800073083120313F6
:100626009F0083169F01FF3083128500E0308316FA
:100636008500FE30831286000E3083168600013058
:1006460083129000C2308316810090308312980086
:1006560024308316980005309900313083129000BB
:1006660004309700343083168C0083128C01E030FE
:100676008B000F3085001B30A200A501C201C3010B
:100686004208383E8400831377308000C20A03197B
:10069600C30A4308803AF000803070020A3003191A
:1006A6004202031C432BB8220038031DE92BFA2B08
:1006B600A501A50A602B0230A500A301FA2BC201F1
:1006C600C3014208383E84008313FF308000C20A0B
:1006D6000319C30A4308803AF000803070020A30DA
:1006E600031942020318FA2B642BC201C301420804
:1006F6002E3E840083138001C20A0319C30A4308ED
:10070600803AF000803070020A3003194202031862
:10071600FA2B7A2BC201C3014208383E84008313A8
:100726008001C20A0319C30A4308803AF0008030E8
:1007360070020A30031942020318FA2B8F2BC201EA
:10074600C30142082E3E84008313FF308000C20A94
:100756000319C30A4308803AF000803070020A3059
:10076600031942020318FA2BA42B03305F2BCA226B
:10077600313A03195B2B033A03195E2B013A03192D
:10078600622B073A0319782B013A03198D2B033A8A
:100796000319A22B013A0319B82BFA2BCA22FF3AE6
:1007A600F0002308383E8400831370088000A30AF3
:1007B60023080A3A031DFA2BE72BCA22F000230866
:1007C6002E3ED62BCA22A200A501FA2B2508F00040
:1007D600043070020318FA2B03308A00F6307007D3
:1007E60003188A0A8200BA2BD12BE02BE52B201D99
:0A07F600562B20112708F622562B7F
:00000001FF
